:020000040000FA
:100000002828820752346F346F346D3420345434CE
:1000100065346D347034203482075334653474345D
:100020002034543465346D347034203482073C34C9
:100030005334653474342034543465346D3470343E
:100040002034463469347234733474343E3420348A
:100050008A2018212030B00005168030B100102110
:10006000A301230816203C21A30A10302302031DFC
:100070003128C530B1001021A8010310300CA80DA3
:10008000A7006821FC20851847286121B00A85193E
:1000900039280130B10010215B21A30123080C2075
:1000A0003C21A30A09302302031D4E28FC20C03046
:1000B000B1001021A301230801203C21A30A09302B
:1000C0002302031D5B28051694202008A8010310B5
:1000D000200CA80DA700682120083002031C7628F8
:1000E000C930B1001021FC20612163280512C930FC
:1000F000B1001021FC20612194202008A8010310E8
:10010000200CA80DA70068212008013E300203182A
:1001100063287628850107309F008316EF3085001D
:100120000630860083120800E320013E031D08000C
:10013000B520031DAF28CC30CC20BE30CC20E3202E
:10014000A000E320A100B520CC30CC204430CC204E
:1001500021080319AE28013E031DAF2800340134E5
:1001600000000000A90BB028080005108316051038
:1001700083127730A900B0208316051483120C3047
:10018000A900B0200000000005080139AA003B309A
:10019000A900B0202A080800AB000830AA0005100A
:1001A0008316051083120130A900B020AB0C031890
:1001B00005140D30A900B020831605148312000029
:1001C000AA0BCF2808000830AA00051083160510D6
:1001D00083120130A900B020831605148312000099
:1001E000000005080139FF3EAB0C0B30A900B02020
:1001F000AA0BE5282B08080026080319E030303E3A
:100200003C212508303E3C212408303E3C212E3044
:100210003C213030281835303C2143303C21080047
:1002200006108611562131083C21861556210800FA
:100230000610861156213830AE0044215121562136
:100240003830AE004421512156213830AE004421CF
:10025000512156213830AE004421512156212830F9
:10026000AE0044215121562128303C210C303C2144
:1002700001303C215B210800AE0044215121AE0E2B
:10028000442151215621080006122E1A0616861204
:10029000AE1A861606132E1B06178613AE1B86177C
:1002A0000800061400000610562108002A30AA0093
:1002B000AA0B582908002930AB005621AB0B5D2949
:1002C0000800AC01AD01AD0B6329AC0B632908003C
:1002D000A5010A302702031C7129A50A0A30A702CA
:1002E00069292708A400A6010A302502031C08007A
:1002F000A60A0A30A5027429FF3FFF3FFF3FFF3FD8
:10030000FF3FFF3FFF3FFF3FFF3FFF3FFF3FFF3FFD
:10031000FF3FFF3FFF3FFF3FFF3FFF3FFF3FFF3FED
:10032000FF3FFF3FFF3FFF3FFF3FFF3FFF3FFF3FDD
:10033000FF3FFF3FFF3FFF3FFF3FFF3FFF3FFF3FCD
:02400E00223F4F
:08400000FF3FFF3FFF3FFF3FC0
:00000001FF
